 cspi

 Timestamp is 4da293a0 (Mon Apr 11 17:37:36 2011)

 Preferred load address is 10000000

 Start         Length     Name                   Class
 0001:00000000 00000004H .CRT$XCA                CODE
 0001:00000004 00000004H .CRT$XCZ                CODE
 0001:00000008 00000004H .CRT$XIA                CODE
 0001:0000000c 00000004H .CRT$XIZ                CODE
 0001:00000010 00000004H .CRT$XPA                CODE
 0001:00000014 00000004H .CRT$XPZ                CODE
 0001:00000018 00000004H .CRT$XTA                CODE
 0001:0000001c 00000004H .CRT$XTZ                CODE
 0001:00000020 00000058H .rdata                  CODE
 0001:00000078 00000021H .rdata$debug            CODE
 0001:0000009c 00002990H .text                   CODE
 0001:00002a2c 00000048H .xdata                  CODE
 0001:00002a74 0000003cH .idata$2                CODE
 0001:00002ab0 00000014H .idata$3                CODE
 0001:00002ac4 000000f8H .idata$4                CODE
 0001:00002bbc 0000013aH .idata$6                CODE
 0001:00002d00 00000100H .edata                  CODE
 0002:00000000 000000f8H .idata$5                DATA
 0002:000000f8 0000000cH .data                   DATA
 0002:00000104 00000010H .bss                    DATA
 0003:00000000 000001f8H .pdata                  DATA

  Address         Publics by Value              Rva+Base       Lib:Object

 0000:00000000       ___safe_se_handler_count   00000000     <absolute>
 0000:00000000       ___safe_se_handler_table   00000000     <absolute>
 0001:00000000       __xc_a                     10001000     corelib0:crt0init.obj
 0001:00000004       __xc_z                     10001004     corelib0:crt0init.obj
 0001:00000008       __xi_a                     10001008     corelib0:crt0init.obj
 0001:0000000c       __xi_z                     1000100c     corelib0:crt0init.obj
 0001:00000010       __xp_a                     10001010     corelib0:crt0init.obj
 0001:00000014       __xp_z                     10001014     corelib0:crt0init.obj
 0001:00000018       __xt_a                     10001018     corelib0:crt0init.obj
 0001:0000001c       __xt_z                     1000101c     corelib0:crt0init.obj
 0001:0000003c       ??_C@_1M@EENNDIOJ@?$AAI?$AAn?$AAd?$AAe?$AAx?$AA?$AA@ 1000103c     cspi_mx25_topaz_v1:cspi_io.obj
 0001:00000048       dmaDriverPath              10001048     ddk_dma:ddk_dma.obj
 0001:00000060       dmaDriverName              10001060     ddk_dma:ddk_dma.obj
 0001:0000009c       BSPCSPICalculateDivRate    1000109c f   bspcspi.obj
 0001:000000e4       BSPCSPISetIOMux            100010e4 f   bspcspi.obj
 0001:000005a4       BSPCSPIReleaseIOMux        100015a4 f   bspcspi.obj
 0001:000005ac       BSPCSPIEnableClock         100015ac f   bspcspi.obj
 0001:000005fc       BSPCspiGetChannelPriority  100015fc f   bspcspi.obj
 0001:00000614       BSPCspiIsDMAEnabled        10001614 f   bspcspi.obj
 0001:0000062c       BSPCspiAcquireGprBit       1000162c f   bspcspi.obj
 0001:00000640       BSPCspiIsAllowPolling      10001640 f   bspcspi.obj
 0001:00000664       BSPCspiExchange            10001664 f   bspcspi.obj
 0001:0000069c       BSPCheckPort               1000169c f   bspcspi.obj
 0001:000006a4       ?SPI_Deinit@@YAHK@Z        100016a4 f   cspi_mx25_topaz_v1:cspi_io.obj
 0001:000006d0       ?SPI_Open@@YAKKKK@Z        100016d0 f   cspi_mx25_topaz_v1:cspi_io.obj
 0001:000006d4       ?SPI_Close@@YAHK@Z         100016d4 f   cspi_mx25_topaz_v1:cspi_io.obj
 0001:000006dc       ?SPI_PowerDown@@YAXK@Z     100016dc f   cspi_mx25_topaz_v1:cspi_io.obj
 0001:000006e0       ?SPI_PowerUp@@YAXXZ        100016e0 f   cspi_mx25_topaz_v1:cspi_io.obj
 0001:000006e4       ?SPI_Read@@YAKKPAXK@Z      100016e4 f   cspi_mx25_topaz_v1:cspi_io.obj
 0001:000006ec       ?SPI_Write@@YAKKPBXK@Z     100016ec f   cspi_mx25_topaz_v1:cspi_io.obj
 0001:000006f4       ?SPI_Seek@@YAKKJG@Z        100016f4 f   cspi_mx25_topaz_v1:cspi_io.obj
 0001:00000704       ?SPI_IOControl@@YAHKKPAEK0KPAK@Z 10001704 f   cspi_mx25_topaz_v1:cspi_io.obj
 0001:00000928       ?SPI_Init@@YAKPBG@Z        10001928 f   cspi_mx25_topaz_v1:cspi_io.obj
 0001:000009dc       ??0cspiClass@@QAA@XZ       100019dc f   cspi_mx25_topaz_v1:cspiClass.obj
 0001:00000a20       ??1cspiClass@@QAA@XZ       10001a20 f   cspi_mx25_topaz_v1:cspiClass.obj
 0001:00000a24       ?CspiRelease@cspiClass@@QAAXXZ 10001a24 f   cspi_mx25_topaz_v1:cspiClass.obj
 0001:00000b40       ?CspiExchangeSize@cspiClass@@AAAIPAUCSPI_XCH_PKT0_T@@@Z 10001b40 f   cspi_mx25_topaz_v1:cspiClass.obj
 0001:00000b94       ?CspiBufRd8@cspiClass@@CAIPAX@Z 10001b94 f   cspi_mx25_topaz_v1:cspiClass.obj
 0001:00000b9c       ?CspiBufRd16@cspiClass@@CAIPAX@Z 10001b9c f   cspi_mx25_topaz_v1:cspiClass.obj
 0001:00000ba4       ?CspiBufRd32@cspiClass@@CAIPAX@Z 10001ba4 f   cspi_mx25_topaz_v1:cspiClass.obj
 0001:00000bac       ?CspiBufWrt8@cspiClass@@CAXPAXI@Z 10001bac f   cspi_mx25_topaz_v1:cspiClass.obj
 0001:00000bb8       ?CspiBufWrt16@cspiClass@@CAXPAXI@Z 10001bb8 f   cspi_mx25_topaz_v1:cspiClass.obj
 0001:00000bc4       ?CspiBufWrt32@cspiClass@@CAXPAXI@Z 10001bc4 f   cspi_mx25_topaz_v1:cspiClass.obj
 0001:00000bcc       ?MapDMABuffers@cspiClass@@QAAHXZ 10001bcc f   cspi_mx25_topaz_v1:cspiClass.obj
 0001:00000c30       ?DeinitChannelDMA@cspiClass@@QAAHXZ 10001c30 f   cspi_mx25_topaz_v1:cspiClass.obj
 0001:00000c6c       ?InitChannelDMA@cspiClass@@QAAHI@Z 10001c6c f   cspi_mx25_topaz_v1:cspiClass.obj
 0001:00000d44       ?InitCspiDMA@cspiClass@@QAAHI@Z 10001d44 f   cspi_mx25_topaz_v1:cspiClass.obj
 0001:00000da4       ?CspiEnableLoopback@cspiClass@@QAAXH@Z 10001da4 f   cspi_mx25_topaz_v1:cspiClass.obj
 0001:00000dbc       ?CheckPort@cspiClass@@QAAHXZ 10001dbc f   cspi_mx25_topaz_v1:cspiClass.obj
 0001:00000dd8       ?CSPI2DataExchange@cspiClass@@QAAHPAUCSPI_XCH_PKT_T@@@Z 10001dd8 f   cspi_mx25_topaz_v1:cspiClass.obj
 0001:00000f0c       ?CspiNonDMADataExchange@cspiClass@@AAAIPAUCSPI_XCH_PKT0_T@@@Z 10001f0c f   cspi_mx25_topaz_v1:cspiClass.obj
 0001:00001484       ?CspiDMADataExchange@cspiClass@@AAAIPAUCSPI_XCH_PKT0_T@@@Z 10002484 f   cspi_mx25_topaz_v1:cspiClass.obj
 0001:00001908       ?CspiEnqueue@cspiClass@@QAAHPAUCSPI_XCH_PKT_T@@@Z 10002908 f   cspi_mx25_topaz_v1:cspiClass.obj
 0001:00001d18       ?CspiProcessQueue@cspiClass@@CAKPAX@Z 10002d18 f   cspi_mx25_topaz_v1:cspiClass.obj
 0001:00001eb8       ?CspiInitialize@cspiClass@@QAAHK@Z 10002eb8 f   cspi_mx25_topaz_v1:cspiClass.obj
 0001:000020d0       CspCSPIGetBaseRegAddr      100030d0 f   cspi_mx25_topaz_v1:cspspi.obj
 0001:0000210c       CspCSPIGetIRQ              1000310c f   cspi_mx25_topaz_v1:cspspi.obj
 0001:0000213c       CspCSPIGetDmaReqTx         1000313c f   cspi_mx25_topaz_v1:cspspi.obj
 0001:0000216c       CspCSPIGetDmaReqRx         1000316c f   cspi_mx25_topaz_v1:cspspi.obj
 0001:0000219c       HalAllocateCommonBuffer    1000319c f   ddk_dma:ddk_dma.obj
 0001:00002260       MmMapIoSpace               10003260 f   ddk_map:ddk_map.obj
 0001:00002328       MmUnmapIoSpace             10003328 f   ddk_map:ddk_map.obj
 0001:0000233c       DDKClockGetFreq            1000333c f   cspddk:CSPDDK.dll
 0001:0000234c       DDKIomuxSelectInput        1000334c f   cspddk:CSPDDK.dll
 0001:0000235c       DDKIomuxSetPadConfig       1000335c f   cspddk:CSPDDK.dll
 0001:0000236c       DDKIomuxSetPinMux          1000336c f   cspddk:CSPDDK.dll
 0001:0000237c       DDKClockSetGatingMode      1000337c f   cspddk:CSPDDK.dll
 0001:0000238c       DDKSdmaCloseChan           1000338c f   cspddk:CSPDDK.dll
 0001:0000239c       DDKSdmaInitChain           1000339c f   cspddk:CSPDDK.dll
 0001:000023ac       DDKSdmaAllocChain          100033ac f   cspddk:CSPDDK.dll
 0001:000023bc       DDKSdmaOpenChan            100033bc f   cspddk:CSPDDK.dll
 0001:000023cc       DDKSdmaGetBufDescStatus    100033cc f   cspddk:CSPDDK.dll
 0001:000023dc       DDKSdmaStartChan           100033dc f   cspddk:CSPDDK.dll
 0001:000023ec       DDKSdmaSetBufDesc          100033ec f   cspddk:CSPDDK.dll
 0001:000023fc       DDKSdmaClearBufDescStatus  100033fc f   cspddk:CSPDDK.dll
 0001:0000240c       HalTranslateSystemAddress  1000340c f   ceddk:CEDDK.dll
 0001:0000241c       KernelIoControl            1000341c f   coredll:COREDLL.dll
 0001:0000242c       DisableThreadLibraryCalls  1000342c f   coredll:COREDLL.dll
 0001:0000243c       RegCloseKey                1000343c f   coredll:COREDLL.dll
 0001:0000244c       RegQueryValueExW           1000344c f   coredll:COREDLL.dll
 0001:0000245c       OpenDeviceKey              1000345c f   coredll:COREDLL.dll
 0001:0000246c       EventModify                1000346c f   coredll:COREDLL.dll
 0001:0000247c       CeOpenCallerBuffer         1000347c f   coredll:COREDLL.dll
 0001:0000248c       CeCloseCallerBuffer        1000348c f   coredll:COREDLL.dll
 0001:0000249c       CeAllocAsynchronousBuffer  1000349c f   coredll:COREDLL.dll
 0001:000024ac       CeFreeAsynchronousBuffer   100034ac f   coredll:COREDLL.dll
 0001:000024bc       DeleteCriticalSection      100034bc f   coredll:COREDLL.dll
 0001:000024cc       InterruptDisable           100034cc f   coredll:COREDLL.dll
 0001:000024dc       HeapDestroy                100034dc f   coredll:COREDLL.dll
 0001:000024ec       CloseHandle                100034ec f   coredll:COREDLL.dll
 0001:000024fc       InterruptDone              100034fc f   coredll:COREDLL.dll
 0001:0000250c       WaitForSingleObject        1000350c f   coredll:COREDLL.dll
 0001:0000251c       Sleep                      1000351c f   coredll:COREDLL.dll
 0001:0000252c       LeaveCriticalSection       1000352c f   coredll:COREDLL.dll
 0001:0000253c       EnterCriticalSection       1000353c f   coredll:COREDLL.dll
 0001:0000254c       HeapFree                   1000354c f   coredll:COREDLL.dll
 0001:0000255c       CreateEventW               1000355c f   coredll:COREDLL.dll
 0001:0000256c       HeapAlloc                  1000356c f   coredll:COREDLL.dll
 0001:0000257c       ReleaseSemaphore           1000357c f   coredll:COREDLL.dll
 0001:0000258c       CreateThread               1000358c f   coredll:COREDLL.dll
 0001:0000259c       InitializeCriticalSection  1000359c f   coredll:COREDLL.dll
 0001:000025ac       InterruptInitialize        100035ac f   coredll:COREDLL.dll
 0001:000025bc       CreateSemaphoreW           100035bc f   coredll:COREDLL.dll
 0001:000025cc       HeapCreate                 100035cc f   coredll:COREDLL.dll
 0001:000025dc       FreePhysMem                100035dc f   coredll:COREDLL.dll
 0001:000025ec       VirtualProtect             100035ec f   coredll:COREDLL.dll
 0001:000025fc       AllocPhysMem               100035fc f   coredll:COREDLL.dll
 0001:0000260c       SetLastError               1000360c f   coredll:COREDLL.dll
 0001:0000261c       VirtualFree                1000361c f   coredll:COREDLL.dll
 0001:0000262c       VirtualCopy                1000362c f   coredll:COREDLL.dll
 0001:0000263c       VirtualAlloc               1000363c f   coredll:COREDLL.dll
 0001:0000264c       DllMain                    1000364c f   corelib0:dllmain.obj
 0001:00002758       _DllMainCRTStartup         10003758 f   corelib0:pegdmain.obj
 0001:00002784       __security_init_cookie     10003784 f   corelib0:seccinit.obj
 0001:000027d0       __security_check_cookie    100037d0 f   corelib0:armsecgs.obj
 0001:000027e0       __gsfailure                100037e0     corelib0:armsecgs.obj
 0001:000028e4       _cexit                     100038e4 f   corelib0:cexit.obj
 0001:000028f4       _initterm                  100038f4 f   corelib0:crt0dat.obj
 0001:00002920       _cinit                     10003920 f   corelib0:crt0dat.obj
 0001:00002980       __crt_ExitProcess          10003980 f   corelib0:exitproc_proxy.obj
 0001:0000298c       ??3@YAXPAX@Z               1000398c f   corelib1:COREDLL.dll
 0001:0000299c       __C_specific_handler       1000399c f   corelib1:COREDLL.dll
 0001:000029ac       memset                     100039ac f   corelib1:COREDLL.dll
 0001:000029bc       ??2@YAPAXI@Z               100039bc f   corelib1:COREDLL.dll
 0001:000029cc       memcpy                     100039cc f   corelib1:COREDLL.dll
 0001:000029dc       _XcptFilter                100039dc f   corelib1:COREDLL.dll
 0001:000029ec       __security_gen_cookie2     100039ec f   corelib1:COREDLL.dll
 0001:000029fc       __report_gsfailure         100039fc f   corelib1:COREDLL.dll
 0001:00002a0c       free                       10003a0c f   corelib1:COREDLL.dll
 0001:00002a1c       TerminateProcess           10003a1c f   coredll:COREDLL.dll
 0001:00002a74       __IMPORT_DESCRIPTOR_CSPDDK 10003a74     cspddk:CSPDDK.dll
 0001:00002a88       __IMPORT_DESCRIPTOR_CEDDK  10003a88     ceddk:CEDDK.dll
 0001:00002a9c       __IMPORT_DESCRIPTOR_COREDLL 10003a9c     coredll:COREDLL.dll
 0001:00002ab0       __NULL_IMPORT_DESCRIPTOR   10003ab0     cspddk:CSPDDK.dll
 0002:00000000       __imp_HalTranslateSystemAddress 10004000     ceddk:CEDDK.dll
 0002:00000004       \177CEDDK_NULL_THUNK_DATA  10004004     ceddk:CEDDK.dll
 0002:00000008       __imp_free                 10004008     corelib1:COREDLL.dll
 0002:0000000c       __imp___report_gsfailure   1000400c     corelib1:COREDLL.dll
 0002:00000010       __imp___security_gen_cookie2 10004010     corelib1:COREDLL.dll
 0002:00000014       __imp__XcptFilter          10004014     corelib1:COREDLL.dll
 0002:00000018       __imp_??2@YAPAXI@Z         10004018     corelib1:COREDLL.dll
 0002:0000001c       __imp_memset               1000401c     corelib1:COREDLL.dll
 0002:00000020       __imp___C_specific_handler 10004020     corelib1:COREDLL.dll
 0002:00000024       __imp_??3@YAXPAX@Z         10004024     corelib1:COREDLL.dll
 0002:00000028       __imp_memcpy               10004028     corelib1:COREDLL.dll
 0002:0000002c       __imp_EnterCriticalSection 1000402c     coredll:COREDLL.dll
 0002:00000030       __imp_KernelIoControl      10004030     coredll:COREDLL.dll
 0002:00000034       __imp_DisableThreadLibraryCalls 10004034     coredll:COREDLL.dll
 0002:00000038       __imp_RegCloseKey          10004038     coredll:COREDLL.dll
 0002:0000003c       __imp_RegQueryValueExW     1000403c     coredll:COREDLL.dll
 0002:00000040       __imp_OpenDeviceKey        10004040     coredll:COREDLL.dll
 0002:00000044       __imp_EventModify          10004044     coredll:COREDLL.dll
 0002:00000048       __imp_CeOpenCallerBuffer   10004048     coredll:COREDLL.dll
 0002:0000004c       __imp_CeCloseCallerBuffer  1000404c     coredll:COREDLL.dll
 0002:00000050       __imp_CeAllocAsynchronousBuffer 10004050     coredll:COREDLL.dll
 0002:00000054       __imp_CeFreeAsynchronousBuffer 10004054     coredll:COREDLL.dll
 0002:00000058       __imp_DeleteCriticalSection 10004058     coredll:COREDLL.dll
 0002:0000005c       __imp_InterruptDisable     1000405c     coredll:COREDLL.dll
 0002:00000060       __imp_HeapDestroy          10004060     coredll:COREDLL.dll
 0002:00000064       __imp_CloseHandle          10004064     coredll:COREDLL.dll
 0002:00000068       __imp_InterruptDone        10004068     coredll:COREDLL.dll
 0002:0000006c       __imp_WaitForSingleObject  1000406c     coredll:COREDLL.dll
 0002:00000070       __imp_Sleep                10004070     coredll:COREDLL.dll
 0002:00000074       __imp_LeaveCriticalSection 10004074     coredll:COREDLL.dll
 0002:00000078       __imp_TerminateProcess     10004078     coredll:COREDLL.dll
 0002:0000007c       __imp_HeapFree             1000407c     coredll:COREDLL.dll
 0002:00000080       __imp_CreateEventW         10004080     coredll:COREDLL.dll
 0002:00000084       __imp_HeapAlloc            10004084     coredll:COREDLL.dll
 0002:00000088       __imp_ReleaseSemaphore     10004088     coredll:COREDLL.dll
 0002:0000008c       __imp_CreateThread         1000408c     coredll:COREDLL.dll
 0002:00000090       __imp_InitializeCriticalSection 10004090     coredll:COREDLL.dll
 0002:00000094       __imp_InterruptInitialize  10004094     coredll:COREDLL.dll
 0002:00000098       __imp_CreateSemaphoreW     10004098     coredll:COREDLL.dll
 0002:0000009c       __imp_HeapCreate           1000409c     coredll:COREDLL.dll
 0002:000000a0       __imp_FreePhysMem          100040a0     coredll:COREDLL.dll
 0002:000000a4       __imp_VirtualProtect       100040a4     coredll:COREDLL.dll
 0002:000000a8       __imp_AllocPhysMem         100040a8     coredll:COREDLL.dll
 0002:000000ac       __imp_SetLastError         100040ac     coredll:COREDLL.dll
 0002:000000b0       __imp_VirtualFree          100040b0     coredll:COREDLL.dll
 0002:000000b4       __imp_VirtualCopy          100040b4     coredll:COREDLL.dll
 0002:000000b8       __imp_VirtualAlloc         100040b8     coredll:COREDLL.dll
 0002:000000bc       \177COREDLL_NULL_THUNK_DATA 100040bc     coredll:COREDLL.dll
 0002:000000c0       __imp_DDKSdmaClearBufDescStatus 100040c0     cspddk:CSPDDK.dll
 0002:000000c4       __imp_DDKSdmaSetBufDesc    100040c4     cspddk:CSPDDK.dll
 0002:000000c8       __imp_DDKSdmaStartChan     100040c8     cspddk:CSPDDK.dll
 0002:000000cc       __imp_DDKSdmaGetBufDescStatus 100040cc     cspddk:CSPDDK.dll
 0002:000000d0       __imp_DDKSdmaOpenChan      100040d0     cspddk:CSPDDK.dll
 0002:000000d4       __imp_DDKSdmaAllocChain    100040d4     cspddk:CSPDDK.dll
 0002:000000d8       __imp_DDKSdmaInitChain     100040d8     cspddk:CSPDDK.dll
 0002:000000dc       __imp_DDKSdmaCloseChan     100040dc     cspddk:CSPDDK.dll
 0002:000000e0       __imp_DDKClockSetGatingMode 100040e0     cspddk:CSPDDK.dll
 0002:000000e4       __imp_DDKIomuxSetPinMux    100040e4     cspddk:CSPDDK.dll
 0002:000000e8       __imp_DDKIomuxSetPadConfig 100040e8     cspddk:CSPDDK.dll
 0002:000000ec       __imp_DDKIomuxSelectInput  100040ec     cspddk:CSPDDK.dll
 0002:000000f0       __imp_DDKClockGetFreq      100040f0     cspddk:CSPDDK.dll
 0002:000000f4       \177CSPDDK_NULL_THUNK_DATA 100040f4     cspddk:CSPDDK.dll
 0002:000000f8       g_hDma                     100040f8     ddk_dma:ddk_dma.obj
 0002:000000fc       __security_cookie          100040fc     corelib0:seccinit.obj
 0002:00000100       __security_cookie_complement 10004100     corelib0:seccinit.obj
 0002:00000104       _exitflag                  10004104     corelib0:cexit.obj
 0002:00000108       __onexitend                10004108     <common>
 0002:0000010c       __onexitbegin              1000410c     <common>
 0002:00000110       _pRawDllMain               10004110     <common>

 entry point at        0001:00002758

 Static symbols

 0001:00002668       _DllMainCRTStartupHelper   10003668 f   corelib0:pegdmain.obj
 0001:00002824       doexit                     10003824 f   corelib0:cexit.obj
